:0600000002005B023AFF62
:03000B0002357645
:030013000235763D
:03001B0002002BB5
:030023000239B3EC
:10002B0032416C636F726E204D634272696465205E
:10003B00496E632E20536372697074204F53202DC9
:10004B002056657273696F6E20362E353320202053
:10005B00C2AF75D0007581567A00122FF2122FFBAA
:10006B0012300412300D75B81075A813787FE4F6B2
:10007B00D8FD758DFD758BFD758C88758A08758916
:10008B00217588047536887535087598C07E007F94
:10009B00409020007400F0A3DEFCDFFA75A080789E
:1000AB0000E2F52C75A0807801E2F52D75A0807823
:1000BB0002E2F52E75A0807803E2F52FD2AFD28C39
:1000CB00D28E122344900000123551FAA3123551EF
:1000DB00FBA3123551FCA3123551B46000400274DE
:1000EB0060FD4C6018A3123551F540A3123551A396
:1000FB00123551F54E90000212231C6017903E40B2
:10010B00122F6C7537287455F599780000D8FDD2ED
:10011B00030201B274AAF599780000D8FDC20390CE
:10012B003E51122F6C122F2A75382890000F123562
:10013B0051A2E7920912336D754520754400754B3A
:10014B0000754A30854E4FE54E6056900020A3A3B4
:10015B00D54FFB75A02E7800854E4F123551F2A36B
:10016B0008123551F2A308B8000205A0D54FEC8553
:10017B004E4F854582854483121487A3A3123551B4
:10018B00540F854B82854A83F0A385824B85834A26
:10019B00854582854483A3A3858245858344D54FBA
:1001AB00D11234101233137A00122FF2122FFB12CA
:1001BB003004123004D29C1201E412023B3001F7DE
:1001CB00C2012003F2123239120C1A1210551211FD
:1001DB00EC1214A91214BE80DE75D0089021007F9A
:1001EB005C7E02E0F5F0A3E0F8A3E0F9686034E58B
:1001FB00F0547FB4000512023C8028B401051204B0
:10020B00D48020B402051202998018B40505120A95
:10021B00688010B40905120B678008B40805120535
:10022B00688000E5822406F5820FDEB775D00022C8
:10023B0022AC83AD828F83898275D00075A0247820
:10024B0000E0FB75F000E425F0F5F00582E5826532
:10025B0008602DE0F208DBEF0582C5F003547FB593
:10026B00F01E858209902400E0FBA3D20A753803A7
:10027B0012150A300B0312323975D00889828006A9
:10028B0075373C75D008E5828C838D82F022858290
:10029B000C85830DE50FC3945C23245BF50B850F55
:1002AB0083850982E030E70FB4F8005007850B8295
:1002BB00758325F00204BA850B82758325E0B49013
:1002CB0000400EB4A0004053B4F0030203720204CA
:1002DB00BA540FB540F8E50904B508030204CD85FF
:1002EB000F83F582E030E7030204BA1582E00509BB
:1002FB00C3943CB420005020902400F5F0E540F06E
:10030B00A37403F0A3E5F0F075D0007BFF902400FD
:10031B00D20A12150A75D0080204BA540FB540AEB2
:10032B00E50904B508030204CD850F83F582E0309F
:10033B00E7030204BA60B41582E00509C3943CB428
:10034B0020005020902400F5F0E540F0A37402F05B
:10035B00A3E5F0F075D0007BFF902400D20A1215B4
:10036B000A75D0080204BAE508C39509B407005012
:10037B00030204A1850F83850982E0B47F4A0582BD
:10038B00E0B47F028003B5403F0582E0B40239053B
:10039B0082E0B47F028008B410028003B4302905D8
:1003AB0082E0B40703020459B4010DE508C39509B3
:1003BB00B4090050690204A1B4060DE508C3950900
:1003CB00B40A0050060204A102048C0582E020E767
:1003DB00F760F5B4210050F0F50B0582E020E7E85B
:1003EB000582E020E7E2F5F00582E020E7DA03542E
:1003FB008045F0F5F0858209902400E540F0A37468
:10040B0028F0A3E50B14F0A3E5F0F075D0007BFF0B
:10041B00902400D20A12150A75D0080204BA05827C
:10042B00E020E75DC3943075F00AA4F5F00582E097
:10043B0020E74EC3943025F075F00AA4F5F0058241
:10044B00E020E73DC3943025F014F5F080090582D8
:10045B00E020E72DC3F5F00582E0B4F7248582098F
:10046B00902400E540F0A37418F0A3E5F0F075D0EC
:10047B00007BFF902400D20A12150A75D0080204E3
:10048B00BA30E7030204B575373C850B82758325BB
:10049B0074F7F00204BA850F83850982E020E70A1E
:1004AB000582E582B508F50204CD8582091509851B
:1004BB000C82850D83E50904F0F5096508600302DC
:1004CB0002A9850C82850D8322AC83AD8275D01079
:1004DB00E508B5090302055D850F83850982E005F3
:1004EB0009B4F5ECA8091509E508C398B405005043
:1004FB000302055D120A11B54045902400F0A3F5E7
:10050B00F0120A11FBB40300503525F0F5F0120A76
:10051B0011602CB440005027F925F0F5F0E92405C3
:10052B00FAE508C39509FEB512004026120A11F030
:10053B00A325F0F5F0D9F5120A11B5F00280087574
:10054B00373C05090204DB753803120A21880902BE
:10055B0004DB75D008E5098C838D82F022AC83AD6A
:10056B008275D010E508B50903020631850F838526
:10057B000982E0B4F1028004050980E88509F005E1
:10058B00F0E508B5F00875D0088C838D8222850FB5
:10059B008385F082E0B4F10280DEB4F202800405C0
:1005AB00F080DEE508B50903020631850F83850966
:1005BB0082E00509B4F10F74011209C775A0207808
:1005CB00C8E4F20205AEB4F2161209EE30E00AC22C
:1005DB00E0C2E11209C702063C75373C0205AEF5D5
:1005EB00F01209EE20E00675373C0205AEF8E5F097
:1005FB00B4F009E8D2E11209C70205AEE830E10B0D
:10060B00C2E11209C7E5F024F0F5F075A02078C817
:10061B00E275A033780028F8E5F0F2E80475A02025
:10062B0078C8F20205AE75D008E5098C838D82F08F
:10063B002275A02078C8E2B40300500675373C023F
:10064B0006DA75A033780028F818E2F5F07900186F
:10065B00E229F918B8FFF9E9B5F002800675373CC5
:10066B000206DA75A03378009020C41209721209C1
:10067B0007B4000675373C0206DAB40121E490207A
:10068B00B4F0A3F0A3F0A3F09020B8F0A3F0A3F084
:10069B00A3F09020BCF0A3F0A3F0A3F08012902065
:1006AB00B41209729020B81209729020BC12097210
:1006BB007900C0129020C8E0FA1AE4F5F0E2F308D2
:1006CB000905F0EAB510F6E5F0F0D0120206DD02EE
:1006DB000631120907B402399020B4E0B4FF1AA313
:1006EB00E0B4FF15A3E0B4FF10A3E0B4FF0B1209B5
:1006FB00EED2E31209C702071C7582B4E0700FA398
:10070B00E0700BA3E07007A3E0B540028003020783
:10071B00E575A03378009020C01209729020C0E0DC
:10072B00A3B40016E0A3B40011E0A3B4000CE0B432
:10073B0004028009B4003B0207E20207E2E2B400C4
:10074B003108E22403FEE2FE08902400E540F0A30A
:10075B00E2F008A3EEB510F890240075D000D20A91
:10076B0075380312150A75D0101209EE30E3090221
:10077B0007E575373C0207E275A02078C412092FF4
:10078B00120907B4021475A02078B812092F75A0AE
:10079B002078B412092F7405F0A3E4F0A37401F0D0
:1007AB00A375A02078C8E2F975A0337800E2F008B1
:1007BB00A3E8B511F875A024780075F000A982E2C2
:1007CB000825F0F5F0E8B511F6E5F0F0A3E50FC359
:1007DB00945CFA091208A502084E9020BCE0700E3A
:1007EB00A3E0700AA3E07006A3E07002805514F03A
:1007FB00B4FF187582BEE014F0B4FF0F7582BDE034
:10080B0014F0B4FF067582BCE014F0E50FC3945CE2
:10081B00F5F0902100E5822408F5827A01E0547FFF
:10082B00B40816E5F0B51202800FAD82AE83AFF0BF
:10083B001208518D828E838FF0E5822408F5820A8F
:10084B00BA02DA0206DA90240075A02078C41209E5
:10085B002F75A02078B412092F75A02078B8120933
:10086B002F75A02078BC12092F75A02078C8E2F94B
:10087B0075A0337800E2F008A3E8B511F875A02451
:10088B00780075F000A982E20825F0F5F0E8B511C3
:10089B00F6E5F0F0A3091208A52290340074F1F0EC
:1008AB00A375A0247800E208B4F007F0A3E4F0A34A
:1008BB00801CB4F10A74F0F0A37401F0A3800FB4A0
:1008CB00F20A74F0F0A37402F0A38002F0A3E8B56F
:1008DB0011D474F2F0A3A98290240075A03478008F
:1008EB00E2F008A3E582B511F775D000902400ABB8
:1008FB0011AA12D20A12301675D01022C082C083F0
:10090B009020C4E0B40016A3E0B40011A3E0B4003F
:10091B000CA3E0B401028007B4020280027400D081
:10092B0083D08222E208601674FDF0A30808E21857
:10093B00F0A3E218F0A3E218F0A3E2F0A322E2087E
:10094B00601174FEF0A308E218F0A3E218F0A3E222
:10095B00F0A322E208600C74FFF0A3E218F0A3E20C
:10096B00F0A322E2F0A322C011E2F9B9FD170808A7
:10097B000808E218F0A3E218F0A3E218F0A3E2F0E3
:10098B000808088033B9FE14E4F0A3080808E2183D
:10099B00F0A3E218F0A3E2F00808801CB9FF10E402
:1009AB00F0A3F0A30808E218F0A3E2F0088009E432
:1009BB00F0A3F0A3F0A3E2F008D01122C009C0828B
:1009CB00C083C0E0E50FC3945CF509902100E5827C
:1009DB002408D509FB2407F582D0E0F0D083D08220
:1009EB00D00922C009C082C083E50FC3945CF5090E
:1009FB00902100E5822408D509FB2407F582E0D07D
:100A0B0083D082D00922C083C082850F838882E085
:100A1B0008D082D0832275D0007BFF902400D20AAD
:100A2B0012150AE513B40002802FB40214E50FC3AC
:100A3B00945CFA850F83850982E516FBD20A123086
:100A4B0016E50FC3945CFA74AA3012027455902405
:100A5B0000F07B01D20A12301675D01022AC83AD98
:100A6B008275D010A809E508C398B40C0050030296
:100A7B000B5C850F83E5092402F582E0B43A028012
:100A8B0066B42D60A809E508C398B417005003029B
:100A9B000B5CE5092416F582E0B40D48902400A800
:100AAB00097919120BBD120BED08791A120BBD1235
:100ABB000BED08791B120BBD120BEDE82406F87930
:100ACB001C120BBD120BED08791D120BBD120BED99
:100ADB0008791E120BBD120BED791FE4120BEDE81A
:100AEB00F5098080020B57E509240BF582E0B40D64
:100AFB005BA809E8F9120BBDB41800504C120A118F
:100B0B00B43A46120BBDB43C00503E120A11B43A33
:100B1B0038120BBDB43C005030753803902400E9FB
:100B2B00F8791C120BBD120BED08791D120BBD12BF
:100B3B000BED08791E120BBD120BED791FE4120B96
:100B4B00EDE509240CF509416F75373C0509020ADF
:100B5B006F75D008E5098C838D82F022AC83AD8252
:100B6B0075D010A809E508C398B405004039850F66
:100B7B0083850982E0B4432AA809E5092403F8E830
:100B8B00120BBD601AB46300501514758330F582D7
:100B9B00E0D2E2F0753803E5092405F50980C47548
:100BAB00373C0509020B6E75D008E5098C838D82E5
:100BBB00F022C083C082850F838882E0080582C340
:100BCB009430B40600501475F00AA4F5F0E008C395
:100BDB009430B40A00500425F0800274FFD082D008
:100BEB008322C0F0F5F0E540F0A37428F0A3E9F000
:100BFB00A3E5F0F0A324282903547FF075D0007BE4
:100C0B00FF902400D20A12150A75D010D0F0229052
:100C1B008000E0F8C52C6830E00CC0E0A26075F0F5
:100C2B0000120E0BD0E030E10CC0E0A26175F001B8
:100C3B00120E0BD0E030E20CC0E0A26275F0021293
:100C4B000E0BD0E030E30CC0E0A26375F003120E84
:100C5B000BD0E030E40CC0E0A26475F004120E0B74
:100C6B00D0E030E50CC0E0A26575F005120E0BD09C
:100C7B00E030E60CC0E0A26675F006120E0BD0E079
:100C8B0030E708A26775F007120E0B908001E0F8B1
:100C9B00C52D6830E00CC0E0A26875F008120E0B91
:100CAB00D0E030E10CC0E0A26975F009120E0BD058
:100CBB00E030E20CC0E0A26A75F00A120E0BD0E035
:100CCB0030E30CC0E0A26B75F00B120E0BD0E030D2
:100CDB00E40CC0E0A26C75F00C120E0BD0E030E50A
:100CEB000CC0E0A26D75F00D120E0BD0E030E60CCF
:100CFB00C0E0A26E75F00E120E0BD0E030E708A22A
:100D0B006F75F00F120E0B908002E0F8C52E683055
:100D1B00E00CC0E0A27075F010120E0BD0E030E1C9
:100D2B000CC0E0A27175F011120E0BD0E030E20C8A
:100D3B00C0E0A27275F012120E0BD0E030E30CC0C3
:100D4B00E0A27375F013120E0BD0E030E40CC0E090
:100D5B00A27475F014120E0BD0E030E50CC0E0A2BB
:100D6B007575F015120E0BD0E030E60CC0E0A276D4
:100D7B0075F016120E0BD0E030E708A27775F0175E
:100D8B00120E0B908003E0F8C52F6830E00CC0E02A
:100D9B00A27875F018120E0BD0E030E10CC0E0A277
:100DAB007975F019120E0BD0E030E20CC0E0A27A8C
:100DBB0075F01A120E0BD0E030E30CC0E0A27B757D
:100DCB00F01B120E0BD0E030E40CC0E0A27C75F0EF
:100DDB001C120E0BD0E030E50CC0E0A27D75F01DAF
:100DEB00120E0BD0E030E60CC0E0A27E75F01E12A6
:100DFB000E0BD0E030E708A27F75F01F120E0B220E
:100E0B00920590257DE07003020F6DF54F754D0037
:100E1B00754C26854D82854C83E0F9A3E0FAA3E05F
:100E2B00A3A385824D85834C89828A83F545C0F0C7
:100E3B0075F002A4F54B85F04AD0F0A3A3123551FF
:100E4B00FBA3123551FCA3123551FDA3123551FEF4
:100E5B00A3123551FFEF547FB5F05EEB20E4052074
:100E6B0005578003300552EE600CB4070050071293
:100E7B000F7140028043903000E5452582F582E0FA
:100E8B0030E23030E02FE54B2400F582E54A343177
:100E9B00F58312149AE582C39CE5839D5003020FE0
:100EAB006AE545122070758330854582E0D2E2F009
:100EBB00020F6AD2E2F0020F6AA3123551FEA3129F
:100ECB003551FFEF547FB5F02BEB20E505200524C2
:100EDB00800330051FEE600CB407005007120F7132
:100EEB0040028010903000E5452582F582E0C2E299
:100EFB00F0020F6AA3123551FEA3123551FFEF54C6
:100F0B007FB5F02BEB20E605200524800330051F71
:100F1B00EE600CB407005007120F71400280109066
:100F2B003000E5452582F582E0D2E3F0020F6AA39B
:100F3B00123551FEA3123551FFEF547FB5F020EB64
:100F4B0020E7052005198003300514EE600CB4076B
:100F5B00005007120F7140028005E545122070D535
:100F6B004F0122020E1EC082C083C0F0E58224070F
:100F7B00F582E5833400F583123551F8A312355110
:100F8B00541F240BF975A025E3F9EE30E708E8545C
:100F9B001F240BF8E2F8EE540F2323900FAA7302D1
:100FAB000FEA00020FEE00020FFC0002100A000213
:100FBB00101A0002102C0002103C00020FEE00026F
:100FCB000FFC0002100A0002101A0002102C000283
:100FDB00103C00020FEA00020FEA00020FEA00C306
:100FEB0002104EE988F0B5F004D302104EC3021084
:100FFB004EE988F0B5F004C302104ED302104EE94F
:10100B0088F0B5F0004004C302104ED302104EE935
:10101B0088F0B5F00280064004C302104ED30210D4
:10102B004EE889F0B5F00040E2C302104ED3021037
:10103B004EE889F0B5F00280064004C302104ED38F
:10104B0002104ED0F0D083D08222200F03021184E5
:10105B0090257EE07003021184F54F754D00754CA1
:10106B002A854D82854C83E0F9A3E0FAA3E0A3A384
:10107B0085824D85834C89828A83F545C0F075F056
:10108B0002A4F54B85F04AD0F0A3A3123551FBA374
:10109B00123551FCA3123551FDA3123551FEA3128B
:1010AB003551FFEE541FB40700404A12118740021E
:1010BB008043903000E5452582F582E030E2303008
:1010CB00E02FE54B2400F582E54A3431F583121409
:1010DB009AE582C39CE5839D5003021170E545128E
:1010EB002070758330854582E0D2E2F0021170D218
:1010FB00E2F0021170A3123551FEA3123551FFEE2F
:10110B00541FB40700401712118740028010903013
:10111B0000E5452582F582E0C2E2F0021170A312D0
:10112B003551FEA3123551FFEE541FB40700401783
:10113B0012118740028010903000E5452582F58220
:10114B00E0D2E3F0021170A3123551FEA312355118
:10115B00FFEE541FB40700400C12118740028005AC
:10116B00E545122070D54F0302117902106C7E20D9
:10117B0090252B7400F0A3DEFCC20F22C082C0832B
:10118B00C0F0E5822407F582E5833400F583123540
:10119B0051F8A3123551541FF990252B2582F58256
:1011AB00E0C2046002D204EE30E719E8541FF89055
:1011BB00252B2582F582E06002D20475A025740BE5
:1011CB0028F8E2F830041275A025740B29F9E3F91D
:1011DB00EE540F2323900FAA73C3D0F0D083D08289
:1011EB0022854E4FE54E7003021445754B00754A30
:1011FB0030754D00754C2E900020E54E12144C8529
:10120B008247858346754300754231754520754489
:10121B0000854B82854A83E020E2030213DB9000BA
:10122B001C1235515401700890001B12355160325D
:10123B0085458285448312148774152582F5827443
:10124B00003583F58312355130E017C082C08320FF
:10125B00E104740080027401903504F0D083D082D5
:10126B008011C082C0837400903504F0D083D0828B
:10127B00021354A3123551F8A3123551F9A31235A9
:10128B0051FA903502E0FB903501E0FC903500E01F
:10129B00FDC3EB98F582EC99F5838542A0A843E555
:1012AB0082F208E583F2ED9A30E703021342707184
:1012BB00903505854FF0C3E58225F0F582E5833443
:1012CB0000F583E020E211E2701718E275F005B526
:1012DB00F002800440028009903503E07003021392
:1012EB006A903504E0700302139B85478285468321
:1012FB00121487858249858348121487E5824583BA
:10130B00601F12145F600A854982854883A3A380FE
:10131B00E2854D82854C83E549F0A3E548F0021345
:10132B00CE903504E06069854D82854C83E549F0AC
:10133B00A3E548F00213CE854782854683121487B6
:10134B008582498583480213CE8543828542831269
:10135B00149AA38542A0A843E582F208E583F2859F
:10136B004D82854C8312149A8582498583481214C9
:10137B0087E5824583601912145F6047A3A3C20AF5
:10138B0012150A20063D854982854883A3A380D880
:10139B00903504E0702D854782854683121487852E
:1013AB0082498583488542A0A8437400F208F285E0
:1013BB004B82854A83E030E10510E3028002C2E2F2
:1013CB00C2E4F0854D82854C83E549F0A3E548F0F6
:1013DB00854B82854A83E0F9903505854FF0C3E54F
:1013EB008225F0F582E5833400F583E9F0D54F02D1
:1013FB008048854B82854A83A385824B85834A85AA
:10140B004D82854C83A3A385824D85834C85478272
:10141B00854683A3A3858247858346854382854280
:10142B0083A3A3858243858342854582854483A319
:10143B00A385824585834402121C9035037400F00A
:10144B0022C0F075F002A42582F582E5F03583F514
:10145B0083D0F022AD82AE83121487AB82AC83852E
:10146B00438285428312149AE582C39BE5839C4099
:10147B000474FF800274008D828E8322C0F01235BB
:10148B0051F5F0A3123551F58385F082D0F022C0CF
:10149B00F0E0F5F0A3E0F58385F082D0F022AA24EA
:1014AB00122FF2AA25122FFBAA26123004AA2712FA
:1014BB00300D22301348E550B4024314F550780038
:1014CB0075A02574FFF208E540F2087400F208E5F8
:1014DB002CF208E52DF208E52EF208E52FF2089024
:1014EB008004E0F208A3E0F208A3E0F208A3E0F224
:1014FB0008A3E0F29025007A007B2B12301622C253
:10150B0006AD82AE837A0012355DFFA312355DC244
:10151B0012B467004003D21222903D4175F002A431
:10152B002582F582E5F03583F583E493F5F0A3E4AA
:10153B009385F083F582E4731216EF0216EA121705
:10154B00570216EA1217BC0216EA12181A0216EA0A
:10155B001218840216EA1218EC0216EA1218FB0291
:10156B0016EA12193A0216EA1219520216EA12195F
:10157B006A0216EA1219930216EA121AEA0216EA1C
:10158B001232DB0216EA121B480216EA121B8F02FA
:10159B0016EA121CB20216EA121DD50216EA121E28
:1015AB000C0216EA121E730216EA121EDA0216EA71
:1015BB00121F4F0216EA121DEA0216EA121FC4028C
:1015CB0016EA12202A0216EA1220430216EA122009
:1015DB005C0216EA1221910216EA1222A20216EA04
:1015EB001224CA0216EA0216EA122F2A0216EA126D
:1015FB002F4A0216EA1225200216EA12254E02166F
:10160B00EA1226520216EA1226760216EA1226A2CF
:10161B000216EA1226CF0216EA1227000216EA1267
:10162B00272F0216EA1227620216EA1227930216D6
:10163B00EA1227CD0216EA1228080216EA122847E8
:10164B000216EA1228840216EA1228C50216EA12BA
:10165B0029040216EA12292B0216EA122954021641
:10166B00EA1229800216EA1229B10216EA1229E4BB
:10167B000216EA122A1B0216EA122A500216EA1264
:10168B002A890216EA122AC00216EA122AFF021649
:10169B00EA122B400216EA122B850216EA122BC80D
:1016AB000216EA122C0F0216EA122C540216EA1238
:1016BB002C830216EA12257C0216EA1225D6021694
:1016CB00EA122CB40216EA122D3D0216EA122D7301
:1016DB000216EA122F140216EA122DB20216EA8D26
:1016EB00828E83228D828E83A3A312355D20E64FDB
:1016FB00122302B900104224F4F5F0902040E0557B
:10170B00F0F052288045B901104225F4F5F09020F5
:10171B0041E055F0F052298032B902104226F4F51F
:10172B00F0902042E055F0F0522A801FB9030E4290
:10173B0027F4F5F0902043E055F0F0522B800C5439
:10174B003F2474F58275832074FFF0228D828E8383
:10175B00A3A312355D20E64C122302F4B9000F52FD
:10176B0024F5F0902040E055F0F052288042B9016A
:10177B000F5225F5F0902041E055F0F052298030C2
:10178B00B9020F5226F5F0902042E055F0F0522AA4
:10179B00801EB9030D5227F5F0902043E055F0F071
:1017AB00522B800C543F2474F5827583207400F007
:1017BB00228D828E83A3A312355DF8541F23240040
:1017CB00C8122302FAA312355D75A020F208F2EAC3
:1017DB00B9000DF5F0902040E045F0F04228802E46
:1017EB00B9010DF5F0902041E045F0F04229801E43
:1017FB00B9020DF5F0902042E045F0F0422A800E40
:10180B00B9030BF5F0902043E045F0F0422B228D0D
:10181B00828E83A3A312355DF8541F232400C812B4
:10182B002302FAA312355D75A020F208F2EAB90083
:10183B001042286224F4F5F0902040E055F0F0803F
:10184B0037B9011042296225F4F5F0902041E0559B
:10185B00F0F08024B90210422A6226F4F5F09020B1
:10186B0042E055F0F08011B9030E422B6227F4F5DC
:10187B00F0902043E055F0F0228D828E83A3A312CB
:10188B00355D20E64F122302B900106224F4F5F007
:10189B00902040E055F0F052288045B901106225A8
:1018AB00F4F5F0902041E055F0F052298032B90266
:1018BB00106226F4F5F0902042E055F0F0522A80A9
:1018CB001FB903106227F4F5F0902043E055F0F0B8
:1018DB00522B800C543F2474F582758320E0F4F076
:1018EB00228D828E83A3A312355DFBA31223A2222A
:1018FB00902200E0F8A3E0F5F075A05E902100E0E7
:10190B00547FB4010579010219177900903E11E952
:10191B0093600BF20908E8B5F0F5D206801090221F
:10192B0000E8C2ACF0200804D208D299D2AC228DC8
:10193B00828E83A3A312355DFAA312355DFBA3122E
:10194B0030166002D206228D828E83A3A312355DE0
:10195B00FAA312355DFBA31230916002D206228DE1
:10196B00828E83A3A312355DFA7B01A312355D90A2
:10197B00250B2582F582A20AC0D0D20A123016D0CE
:10198B00D0920A6002D206228D828E83A3A31235D7
:10199B005DFAA312355DC0E0A312355DFF5407233A
:1019AB00239019B0730219CF00021A0100021A2CEE
:1019BB0000021A51000219CF000219CF000219CFF1
:1019CB00000219CFD0E090250B2582F582E078003C
:1019DB0079007C00600F75F00A84A8F0600775F041
:1019EB000A84A9F0FCE82430F8E92430F9EC24301F
:1019FB00FC7B03021A6FD0E090250B2582F582E069
:101A0B00540F2430B43A0040022407F9E054F0C4D8
:101A1B002430B43A0040022407FC78207B02021ADF
:101A2B006FD0E090250B2582F582E054072430F827
:101A3B00E054380303032430F9E054C0232324304B
:101A4B00FC7B03021A6FD0E090250B2582F5827B7D
:101A5B0001A20AC0D0D20A123016D0D0920A607EF0
:101A6B00D206807AEF543803901A7773021A9600D5
:101A7B00021ACA00021ABB00021AA400021A96002C
:101A8B00021A9600021A9600021A96BB0102802FC8
:101A9B00BC302CE9FCE8F9DBF2BC3023E9FCE8F9BB
:101AAB007820BB031ABC3017E9FCE8F97820800FCB
:101ABB00BC300C7C20BB0307B9300479208000902C
:101ACB002044ECF0A3E9F0A3E8F0902044A20AC074
:101ADB00D0D20A123016D0D0920A6002D206228DD2
:101AEB00828E83A3A312355DFAA312355DF8A31280
:101AFB00355DF9A312355D90250B2582F582E0FB50
:101B0B009020447406F0A3E5404480F0FCA3E8F079
:101B1B002CFCA37428F02CFCA3E9F02CFCA3EBF019
:101B2B002CA303547FF09020447B07A20AC0D0D291
:101B3B000A123016D0D0920A6002D206228D828E03
:101B4B008375D010A3A312355DFBA3AD82AE83903A
:101B5B002100E5822408F5827A01E0547FB408194C
:101B6B00A882A9838D828E8375D000AA12AB131223
:101B7B00301675D01088828983E5822408F5820A95
:101B8B00BA02D722854B82854A83E0F98D828E83F8
:101B9B00A3A312355DFA232323FC75A021F8E920BA
:101BAB00E442E2C2E7F2E408F208F2A312355DFB6D
:101BBB00A312301675A021ECF8E2D2E7F208080860
:101BCB00080812355DF2A30812355DF2200606A354
:101BDB000812355DF2854B82854A83E0D2E4F0D260
:101BEB0006021CB108A312355D24052582F582E49B
:101BFB003583F58312355DF5F0E2C395F0501E0881
:101C0B00080808E2F5F008E245F0602D18E2C394ED
:101C1B0001F2500408E214F2D206021CB1ABF0A39D
:101C2B00EA245CF5A0780012355DF5F0E2B5F00919
:101C3B00A308DBF3753803804A75A021EC2407F861
:101C4B00E2600F14F28D828E83A3A3ECF8D206020E
:101C5B001BAD75373C30092B900014123551F8A38E
:101C6B00123551F5838882E5822AF582E43583F5B6
:101C7B0083123551F8C3954E50097583308882E035
:101C8B00D2E2F075A021ECF8E2547FB4030280039A
:101C9B00B40704C2E78002D2E7F2854B82854A8300
:101CAB00E0C2E4F0C20622854B82854A83E0F98DBF
:101CBB00828E83A3A312355DFA232323FC75A02107
:101CCB00F8E920E442E2C2E7F2E408F208F2A312D8
:101CDB00355DFBA312309175A021ECF8E2D2E7F24F
:101CEB00080808080812355DF2A30812355DF220CA
:101CFB000606A30812355DF2854B82854A83E0D236
:101D0B00E4F0D206021DD408A312355D240525820A
:101D1B00F582E43583F58312355DF5F0E2C395F07A
:101D2B00501E08080808E2F5F008E245F0602D188F
:101D3B00E2C39401F2500408E214F2D206021DD45D
:101D4B00ABF0A3EA245CF5A0780012355DF5F0E268
:101D5B00B5F009A308DBF3753803804A75A021ECB5
:101D6B002407F8E2600F14F28D828E83A3A3ECF8A4
:101D7B00D206021CD075373C30092B90001412355B
:101D8B0051F8A3123551F5838882E5822AF582E456
:101D9B003583F583123551F8C3954E500975833051
:101DAB008882E0D2E2F075A021ECF8E2547FB40314
:101DBB00028003B40704C2E78002D2E7F2854B82AC
:101DCB00854A83E0C2E4F0C206228D828E83A3A3F0
:101DDB0012355D547F232549F54950020548228D64
:101DEB00828E83A3A312355DFAA312355DF9EAC384
:101DFB0033FAE933F9EAC32549F549E93548F5489A
:101E0B00228D828E83A3A312355D20E72A10E61C58
:101E1B00122302B9000478248039B9010478258093
:101E2B0032B902047826802B782780272474F87522
:101E3B00A020E270238030547F122302B900047873
:101E4B002C8010B90104782D8009B90204782E80FA
:101E5B0002782F567002800FA312355D547F232515
:101E6B0049F54950020548228D828E83A3A3123572
:101E7B005D20E72A10E61C122302B90004782480A7
:101E8B0039B9010478258032B902047826802B7881
:101E9B002780272474F875A020E260238030547FBC
:101EAB00122302B90004782C8010B90104782D801C
:101EBB0009B90204782E8002782F566002800FA396
:101ECB0012355D547F232549F54950020548228D73
:101EDB00828E83A3A312355D20E72A10E61C122302
:101EEB0002B9000478248039B9010478258032B90D
:101EFB0002047826802B782780272474F875A0207D
:101F0B00E27023803E547F122302B90004782C80A8
:101F1B0010B90104782D8009B90204782E8002785B
:101F2B002F567002801DA312355DFAA312355DF991
:101F3B00EAC333FAE933F9EAC32549F549E9FA3536
:101F4B0048F548228D828E83A3A312355D20E72AA4
:101F5B0010E61C122302B9000478248039B901045D
:101F6B0078258032B902047826802B7827802724A5
:101F7B0074F875A020E26023803E547F122302B9CF
:101F8B000004782C8010B90104782D8009B9020463
:101F9B00782E8002782F566002801DA312355DFAD1
:101FAB00A312355DF9EAC333FAE933F9EAC32549DC
:101FBB00F549E9FA3548F548228D828E83A3A312A1
:101FCB00355DF8C3954E50567583308882E030E20C
:101FDB004A30E04AC004C005900020E812144C12AD
:101FEB001487A3A3A3123551FCA3123551FDE8C0EE
:101FFB00F075F002A42400F582E5F03431F583D0BE
:10200B00F012149AE582C39CE5839DD005D0044061
:10201B000DE81220707583308882E0D2E2F0228DB9
:10202B00828E83A3A312355DF8C3954E5009758339
:10203B00308882E0C2E2F0228D828E83A3A3123518
:10204B005DF8C3954E50097583308882E0D2E3F07A
:10205B00228D828E83A3A312355DF8C3954E500457
:10206B00E812207022C000C003C004C0F0F890003A
:10207B0020E54E12144CE812144C121487AB82ACB0
:10208B008375832EE875F002A4F582E5F03583F5B0
:10209B0083EBF0A3ECF0758331E875F002A4F582C5
:1020AB00E5F03583F583E4F0A3F07583308882E0A7
:1020BB00C2E2C2E4F0C2E3D0F0D004D003D00022DD
:1020CB00902200E0F875A05E902100E0547FB400F0
:1020DB00047402F208900002123551A3F208123573
:1020EB0051F208902200E8C2ACF0200804D208D2CA
:1020FB0099D2AC22C004C005C00675A025784B79D7
:10210B001075040075050075060CD5041DD5051A50
:10211B00D506177455C29BC299F5997504007505C0
:10212B0004D504FDD505FA02005B3098DDE599F284
:10213B00C298EA70011B1AEB7003EA601108D9C14F
:10214B00784B7910E2123541A308D9F880AC7A00AC
:10215B007B20DAFEDBFC784B7910E2123541A308C9
:10216B00D9F8902100E0547FB4011474AAC29BC229
:10217B0099F599750400750508D504FDD505FAD0B8
:10218B0006D005D00422C2AF8D828E83A3A3123555
:10219B005DFAA312355DFBE599C29874AAC29BC286
:1021AB0099F5999000001220FF02005B8D828E83BF
:1021BB00A3A312355DFAA312355DFB900002123515
:1021CB0051F8A3123551C854F0241CC8500104F522
:1021DB00838882745A123541A374A5123541A3EA40
:1021EB00123541A3EB123541A3C000C001750000AD
:1021FB00750100D500FDD501FAD001D000C2AFE5C5
:10220B0099C29874AAC29BC299F5991220FF74AA1D
:10221B00C29BC299F599750400750504D504FDD5CB
:10222B0005FA02005B2014FDC29BD214F599229093
:10223B000002123551F8A3123551C854F0241CC8B2
:10224B00500104F5838882123551B45A18A3123504
:10225B0051B4A511A3123551FAA3123551FBA3BAF0
:10226B00000CBB0009E4122230122230801AEA1251
:10227B002230EB122230123551A31222301ABAFF40
:10228B00011BBA00F1BB00EE750400750504D50403
:10229B00FDD505FA02005B900002123551FAA3122C
:1022AB003551FB700CEA7009E41222301222308097
:1022BB00278A828B83A3A3AA82AB83EA122230EBF9
:1022CB00122230900000123551A31222301ABAFF9D
:1022DB00011BBA00F1BB00EE750400750504D504B3
:1022EB00FDD505FA02005B8D828E83A3A312355DAB
:1022FB00C2136002D21322F95407C9030303540318
:10230B00C0E07401B90002800323D9FDF9D0E0C904
:10231B00227800790012355128500109F8A3DC0509
:10232B00BD00F28006BCFFED1D80EAE86A7007E98C
:10233B006B7003E4800274FF2290000075A0987804
:10234B0002E230E70BA3E583B405F6C2110223A129
:10235B00D2117A30122F907A30122F907A38122FA6
:10236B00907A80122F907A06122F907A0C122F905F
:10237B007A01122F907A40122F907A5A122FAF7A3D
:10238B0040122F90122FD1B45AC1903E2F122F6CA6
:10239B00903E1E122F7E22EB60627A80122F9012DB
:1023AB00355DB404005029A3DB028050B400047ADD
:1023BB00808010B401047AC08009B402047A94803E
:1023CB00027AD412355DA3543F2AFA122F90802A39
:1023DB00B40C08A37A01122F90801FB40D03A380B5
:1023EB0014B40A03A3800EB40E2EDB11800EFA1266
:1023FB002FAFA380057AC0122F90DBA322A3123537
:10240B005D14A3C082C08390250B2582F582E0D09A
:10241B0083D08212248680E2B40FD3DB0280DDA34B
:10242B0012355D14A3C082C08390250B2582F582E3
:10243B00E0D083D08212244580C07C017A20C394E3
:10244B0064400C1C7A31C394644004C394640A2422
:10245B0064C0E0122FAFD0E07A31C3940A40030A74
:10246B0080F81A240AC0E0BA3005EC60027A201218
:10247B002FAFD0E02430FA122FAF227C017A20C389
:10248B009464400C1C7A31C394644004C394640A72
:10249B002464BA20028007C0E0122FAFD0E07A315B
:1024AB00C3940A40030A80F81A240AC0E0BA300326
:1024BB00EC7003122FAFD0E02430FA122FAF228D25
:1024CB00828E83A3A312355D5403FB7005903E628D
:1024DB008013B40105903E72800BB40205903E82CE
:1024EB008003903E927A01122F907C10E493FA12A3
:1024FB002FAFA3DCF77C107AC0122F90EBC424749F
:10250B00F582758320E060047A3180027A30122FD5
:10251B00AFA3DCF1228D828E83A3A312355DFAA3C8
:10252B0012355DFBEA4224F4F5F0902040E055F0C3
:10253B00F05228EB4225F4F5F0902041E055F0F0F5
:10254B005229228D828E83A3A312355DFAA31235F5
:10255B005DFBEAF45224F5F0902040E055F0F05288
:10256B0028EBF45225F5F0902041E055F0F052297C
:10257B00228D828E83A3A312355DFAA312355DFBE8
:10258B00EA7011EBF524F4F5F0902040E055F0F0F3
:10259B0052288036B4010FEBF525F4F5F09020416D
:1025AB00E055F0F05229B4020FEBF526F4F5F0905C
:1025BB002042E055F0F0522AB4030FEBF527F4F567
:1025CB00F0902043E055F0F0522B228D828E83A3A6
:1025DB00A312355DFAA312355DFBEA701875A025C1
:1025EB00740B2BF8E52CF275A025742B2BF874FFCC
:1025FB00F2D20F8051B4011875A025740B2BF8E59E
:10260B002DF275A025742B2BF874FFF2D20F8036A8
:10261B00B4021875A025740B2BF8E52EF275A025C6
:10262B00742B2BF874FFF2D20F801BB4031875A018
:10263B0025740B2BF8E52FF275A025742B2BF87452
:10264B00FFF2D20F8000228D828E83A3A312355D01
:10265B00541FF9240BF8A312355D75A025F275A054
:10266B0025742B29F874FFF2D20F228D828E83A34F
:10267B00A312355D541FF9240BF875A025E2F5F074
:10268B00A312355DB5F00FA312355D547F23254999
:10269B00F54950020548228D828E83A3A312355D26
:1026AB00541F240BF875A025E2F5F0A312355DB588
:1026BB00F002800FA312355D547F232549F5495055
:1026CB00020548228D828E83A3A312355D541F24ED
:1026DB000BF875A025E2F5F0A312355DC5F0B5F04A
:1026EB00004002800FA312355D547F232549F54925
:1026FB0050020548228D828E83A3A312355D541F91
:10270B00240BF875A025E2F5F0A312355DB5F000AA
:10271B004002800FA312355D547F232549F54950A4
:10272B00020548228D828E83A3A312355D541F248C
:10273B000BF875A025E2F5F0A312355DC5F0B5F0E9
:10274B000280044002800FA312355D547F2325497C
:10275B00F54950020548228D828E83A3A312355D65
:10276B00541F240BF875A025E2F5F0A312355DB5C7
:10277B00F00280044002800FA312355D547F2325A5
:10278B0049F54950020548228D828E83A3A3123549
:10279B005D541FF9240BF875A025E2F5F0A3123553
:1027AB005DB5F01DA312355DFAA312355DF9EAC3D1
:1027BB0033FAE933F9EAC32549F549E9FA3548F51E
:1027CB0048228D828E83A3A312355D541F240BF8F0
:1027DB0075A025E2F5F0A312355DB5F002801DA3BF
:1027EB0012355DFAA312355DF9EAC333FAE933F911
:1027FB00EAC32549F549E9FA3548F548228D828E19
:10280B0083A3A312355D541F240BF875A025E2F5A5
:10281B00F0A312355DC5F0B5F0004002801DA31288
:10282B00355DFAA312355DF9EAC333FAE933F9EAF8
:10283B00C32549F549E9FA3548F548228D828E833F
:10284B00A3A312355D541F240BF875A025E2F5F0F8
:10285B00A312355DB5F0004002801DA312355DFA61
:10286B00A312355DF9EAC333FAE933F9EAC3254913
:10287B00F549E9FA3548F548228D828E83A3A312D8
:10288B00355D541F240BF875A025E2F5F0A3123526
:10289B005DC5F0B5F00280044002801DA312355DCA
:1028AB00FAA312355DF9EAC333FAE933F9EAC32522
:1028BB0049F549E9FA3548F548228D828E83A3A361
:1028CB0012355D541F240BF875A025E2F5F0A31209
:1028DB00355DB5F00280044002801DA312355DFA10
:1028EB00A312355DF9EAC333FAE933F9EAC3254993
:1028FB00F549E9FA3548F548228D828E83A3A31258
:10290B00355D541FF9240BF875A025E2FAA3123597
:10291B005D2AF275A025742B29F974FFF3D20F22CF
:10292B008D828E83A3A312355D541FF9240BF8758A
:10293B00A025E2FAA312355DCAC39AF275A02574DD
:10294B002B29F974FFF3D20F228D828E83A3A3124E
:10295B00355D541FF5F0240BF8A312355D541F247D
:10296B000BF975A025E3F275A025742B25F0F874EF
:10297B00FFF2D20F228D828E83A3A312355D541FDB
:10298B00240BF875A025E2F5F0A312355D541F2436
:10299B000BF9E3B5F00FA312355D547F232549F5F1
:1029AB004950020548228D828E83A3A312355D54B4
:1029BB001F240BF875A025E2F5F0A312355D541F0B
:1029CB00240BF9E3B5F00280DCA312355D547F23B1
:1029DB002549F54950020548228D828E83A3A31207
:1029EB00355D541F240BF875A025E2F5F0A31235C5
:1029FB005D541F240BF9E3C5F0B5F0004002800FC6
:102A0B00A312355D547F232549F549500205482211
:102A1B008D828E83A3A312355D541F240BF875A0F2
:102A2B0025E2F5F0A312355D541F240BF9E3B5F045
:102A3B00004002800FA312355D547F232549F549D1
:102A4B0050020548228D828E83A3A312355D541F3D
:102A5B00240BF875A025E2F5F0A312355D541F2465
:102A6B000BF9E3C5F0B5F00280044002800FA3120E
:102A7B00355D547F232549F54950020548228D8247
:102A8B008E83A3A312355D541F240BF875A025E28A
:102A9B00F5F0A312355D541F240BF9E3B5F002805A
:102AAB00044002800FA312355D547F232549F5495D
:102ABB0050020548228D828E83A3A312355D541FCD
:102ACB00240BF875A025E2F5F0A312355D541F24F5
:102ADB000BF9E3B5F01DA312355DFAA312355DF9C1
:102AEB00EAC333FAE933F9EAC32549F549E9FA357B
:102AFB0048F548228D828E83A3A312355D541F2483
:102B0B000BF875A025E2F5F0A312355D541F240BCD
:102B1B00F9E3B5F00280DCA312355DFAA312355D43
:102B2B00F9EAC333FAE933F9EAC32549F549E9FA76
:102B3B003548F548228D828E83A3A312355D541F31
:102B4B00240BF875A025E2F5F0A312355D541F2474
:102B5B000BF9E3C5F0B5F0004002801DA312355D03
:102B6B00FAA312355DF9EAC333FAE933F9EAC3255F
:102B7B0049F549E9FA3548F548228D828E83A3A39E
:102B8B0012355D541F240BF875A025E2F5F0A31246
:102B9B00355D541F240BF9E3B5F0004002801DA3F3
:102BAB0012355DFAA312355DF9EAC333FAE933F94D
:102BBB00EAC32549F549E9FA3548F548228D828E55
:102BCB0083A3A312355D541F240BF875A025E2F5E2
:102BDB00F0A312355D541F240BF9E3C5F0B5F002D9
:102BEB0080044002801DA312355DFAA312355DF9F6
:102BFB00EAC333FAE933F9EAC32549F549E9FA356A
:102C0B0048F548228D828E83A3A312355D541F2471
:102C1B000BF875A025E2F5F0A312355D541F240BBC
:102C2B00F9E3B5F00280044002801DA312355DFA72
:102C3B00A312355DF9EAC333FAE933F9EAC325493F
:102C4B00F549E9FA3548F548228D828E83A3A31204
:102C5B00355D541FF5F0240BF875A025E2FAA3128D
:102C6B00355D541F240BF9E32AF275A025742B252F
:102C7B00F0F874FFF2D20F228D828E83A3A312354C
:102C8B005D541FF5F0240BF875A025E2FAA312355D
:102C9B005D541F240BF9E3CAC39AF275A025742B5C
:102CAB0025F0F874FFF2D20F228D828E83A3A3122C
:102CBB00355D541FF9903EA27A01122F907C10E4DF
:102CCB0093FA122FAFA3DCF77AC0122F9090240047
:102CDB007420F0A3F0A3F0A3F0A3E904122EACEB45
:102CEB00B430027420F0A3EAF0A37420F0A3743D77
:102CFB00F0A37420F0A375A025E9240BF9E3122EA1
:102D0B00ACECD204B43004C2047420F0A3EBB430A6
:102D1B00052004027420F0A3EAF0A37420F0A3F0C2
:102D2B00A3F0A3F07C10902400E0FA122FAFA3DCE9
:102D3B00F8228D828E83A3A312355D541FF9FB7588
:102D4B00A025240BF9E3FA90001A123551C3940114
:102D5B00B408005012C423441FF583EB44E0F58202
:102D6B00EA123541122F1F228D828E83A3A31235B7
:102D7B005D541FF990001A123551C39401B4080029
:102D8B005024C423441FF583E944E0F582123551E6
:102D9B00FA75A025740B29F8EAF275A025742B2976
:102DAB00F874FFF2D20F22C0F08D828E83A3A31290
:102DBB00355D75F03CA4FEAFF0A312355DC32EFE5E
:102DCB00EF3400FFA312355D75F03CFB7C007D00FA
:102DDB00C3EB2EFBEC3FFCED3400FD15F0E5F07082
:102DEB00EFA312355DF879007A0090000912355186
:102DFB00B4000575F0188013B4030575F019800B3A
:102E0B00B4010575F01E800375F01EC3E82BF8E9BD
:102E1B003CF9EA3DFA15F0E5F070F0900009123537
:102E2B0051B4013AEF700BEE6034B40A03022E3D3D
:102E3B004018C3EE940AFEEF9400FFC3E89412F817
:102E4B00E99400F9EA9400FA80DAC3EE9401FEC328
:102E5B00E89402F8E99400F9EA9400FA80C69035F8
:102E6B0000E0FD903501E0FC903502E0FBC3E89BF0
:102E7B00FFE99C7014EA9D701090001B123551F500
:102E8B00F0EFB5F002800840069035037401F09026
:102E9B003500EAF0903501E9F0903502E8F0D0F01A
:102EAB00227A007B007C00601675F00A84AAF06021
:102EBB000E75F00A84ABF0600675F00A84ACF0EA8C
:102ECB002430FAEB2430FBEC2430FC22900000126F
:102EDB003551FB902000123551FDEBF412354112A8
:102EEB002F1F123551F4B5030E900000123551B55A
:102EFB0003057A18022F047A08902000ED12354151
:102F0B00122F1F90257FEAF022122ED790257FE0FB
:102F1B00FAF599227C0075F032DCFED5F0FB227AB3
:102F2B0080122F907B28902580122FD1F0A3DBF9F4
:102F3B007AC0122F907B28122FD1F0A3DBF9227AC3
:102F4B0080122F907B28902580E0FA122FAFA3DB05
:102F5B00F87AC0122F907B28E0FA122FAFA3DBF880
:102F6B00227A80122F907400936007FA122FAFA36E
:102F7B0080F4227AC0122F907400936007FA122FFC
:102F8B00AFA380F422C0F030111775F00075A09834
:102F9B007802E230E70700D5F0F3022FAC7800EAB5
:102FAB00F2D0F022C0F030111A75F00075A09878AD
:102FBB0002E230E70700D5F0F3022FCE75A0987828
:102FCB0001EAF2D0F022C0F030111975F00075A0B3
:102FDB00987802E230E70700D5F0F3022FEF75A0E7
:102FEB00987803E2D0F02275A0807804EAF4F222FC
:102FFB0075A0807805EAF4F22275A0807806EAF4D1
:10300B00F22275A0807807EAF4F222AE82AF8390A9
:10301B002200EA2323232582F58274003583F5836E
:10302B00E0F8A3E0F9EA245EF5A089F08E828F83A5
:10303B0012355DF2A308E8B5F00302308ADBF1AE7E
:10304B0082AF83902200EA2323232582F58274002A
:10305B003583F583E8BA000FC2ACF0200804D20820
:10306B00D299D2AC023084D20BF0902064EA145483
:10307B000F2582F582E0D2E7F0E48E828F832274F3
:10308B00FF8E828F8322AE82AF83902200EA2323AE
:10309B00232582F58274003583F583E0F8A3E0F9EC
:1030AB00EA245EF5A089F08E828F8312355DB4F32E
:1030BB0008DB1C0BA3E8023144B4F408DB330BA38D
:1030CB00E8023144B4F56EDB4A0BA3E8023144A3AA
:1030DB0012355DB4F30302314014A3C082C0839058
:1030EB00250B2582F582E0D083D08212319A0231F2
:1030FB0044A312355DB4F40302314014A3C082C063
:10310B008390250B2582F582E0D083D0821231EBA0
:10311B00023144A312355DB4F50302314014A3C050
:10312B0082C08390250B2582F582E0D083D082125A
:10313B003196023144123196A3B5F00602318F025B
:10314B0030B6DBFBAE82AF83902200EA232323252C
:10315B0082F58274003583F583E8BA000FC2ACF0B8
:10316B00200804D208D299D2AC023189D20BF0904C
:10317B002064EA14540F2582F582E0D2E7F0E48E46
:10318B00828F832274FF8E828F8322F208E8227F44
:10319B00017E20C39464400C1F7E31C394644004B1
:1031AB00C394640E2464BE2002800EC0E0EE123184
:1031BB0096B5F0030231EAD0E07E31C3940A4003A6
:1031CB000E80F81E240AC0E0BE3003EF700AEE1228
:1031DB003196B5F0030231EAD0E024301231962259
:1031EB007F017E30C39464400C1F7E31C3946440D6
:1031FB0004C394640E2464C0E0EE123196B5F00360
:10320B00023238D0E07E31C3940A40030E80F81EA0
:10321B00240AC0E0BE3005EF60027E30EE1231961C
:10322B00B5F003023238D0E0243012319622200B55
:10323B00030232DA900012123551F5F0A312355118
:10324B00F58385F082A3E5822411F582E5833400B2
:10325B00F583AE82AF8390206475A0907A00C08214
:10326B00C0838E828F8312355154E0B4E007D08334
:10327B00D0820232C2D083D082E030E73AC2E7F08C
:10328B00EAC4032402F8C082C0838E828F83123576
:10329B0051B40A168FF07465F27FD7C2AFDFFE749C
:1032AB0075F27F24DFFED2AFAFF0D083D08274A54E
:1032BB00F20808087406F2A3C082C0838E828F8343
:1032CB00A3AE82AF83D083D0820ABA0191C20B2204
:1032DB008D828E83A3A312355D14540FC40375A086
:1032EB00902402F8A312355DF9C2AF7465F274A590
:1032FB00F27FDEE9DFFED9FCF97475F27F6FDFFE3A
:10330B00D9FC74B5F2D2AF2290000A123551601677
:10331B00758C00758A00D2A9D2AA7530FFF5348559
:10332B003433D2078039C207900009123551B400EB
:10333B000875366A753508801CB4010875368775B3
:10334B0035E98011B403087536707535088006753C
:10335B00368875350885368C85358AC2AAD2A9D2AE
:10336B000222E54E700302340F854E4F7A007B002C
:10337B007800792A7D0075F0267545207544008507
:10338B004582854483121487AE82AF8374052582F0
:10339B00F58274003583F5837C04C204C2051235B3
:1033AB0051A36002D204123551A3B4FF028002D2A2
:1033BB0005DCEB30041788828983EEF0A3EFF0A3D2
:1033CB00E54EC3954FF0A3A3A882A9830B30051933
:1033DB008D8285F083EEF0A3EFF0A3E54EC3954FFE
:1033EB00F0A3A3AD828583F00A854582854483A330
:1033FB00A3858245858344D54F8590257EEBF09040
:10340B00257DEAF022C2A878087A007B0190001291
:10341B00123551F5F0A3123551F58385F082A312C5
:10342B003551F523A3AE82AF83E5822410F582E5F7
:10343B00833400F583123551FD75A021BD00067450
:10344B0000D2E78055BD05067402D2E7804CBD065D
:10345B00067402D2E78043BD0C067401D2E7803AB2
:10346B00BDE0067404D2E78031BD0D067405D2E7CA
:10347B008028BD11067409D2E7801FBD0E067407A4
:10348B00C2E78016BD0F067406D2E7800DBD10068D
:10349B007408D2E780047403C2E7F2FCE82402F953
:1034AB0075A022ECF3BDE00302352375A090EA244E
:1034BB0000F909097410F319197402A21EB392E0F2
:1034CB00BD00028003BD0E0444188011A21BB392F1
:1034DB00E4A21C92E2A21D5004C2E4D2E3F37407EF
:1034EB00301F02740FF3EA2401F9903539E52354A8
:1034FB0007FC93F3EA2404F97488BC06028008BD28
:10350B0005028003BD06027408F3EA2402F9740174
:10351B00F3EA2405F97404F38F838E82E82408F808
:10352B00EA2408FADB02800302342AD2A82244667A
:10353B008899BBCCCCBBC083C0E0E58324A0F583CA
:10354B00D0E0F0D08322C083E58324A0F583E0D0C4
:10355B008322300D04E4938011300A03E0800BC00A
:10356B0083E58324A0F583E0D08322C0D0C0E0C0E4
:10357B0083C08275D010D55003755010E538B40058
:10358B0004D2B480041538C2B4E537B40004D2B504
:10359B0080041537C2B5300005D54102C200E528BD
:1035AB0070030236A030401B902001E014F0701322
:1035BB00C240B220902040E030E008902000E0A311
:1035CB00F0D24030411B902003E014F07013C24145
:1035DB00B221902040E030E108902002E0A3F0D22D
:1035EB004130421B902005E014F07013C242B2220E
:1035FB00902040E030E208902004E0A3F0D242306B
:10360B00431B902007E014F07013C243B2239020A9
:10361B0040E030E308902006E0A3F0D24330441B97
:10362B00902009E014F07013C244B224902040E0C3
:10363B0030E408902008E0A3F0D24430451B9020E2
:10364B000BE014F07013C245B225902040E030E53A
:10365B000890200AE0A3F0D24530461B90200DE0E5
:10366B0014F07013C246B226902040E030E608906A
:10367B00200CE0A3F0D24630472290200FE014F04C
:10368B00701AC247B227902040E030E70F90200E0F
:10369B00E0A3F0D247E529700302379730481B901F
:1036AB002011E014F07013C248B228902041E03092
:1036BB00E008902010E0A3F0D24830491B90201373
:1036CB00E014F07013C249B229902041E030E108B8
:1036DB00902012E0A3F0D249304A1B902015E01441
:1036EB00F07013C24AB22A902041E030E2089020D9
:1036FB0014E0A3F0D24A304B1B902017E014F0706B
:10370B0013C24BB22B902041E030E308902016E01F
:10371B00A3F0D24B304C1B902019E014F07013C265
:10372B004CB22C902041E030E408902018E0A3F03C
:10373B00D24C304D1B90201BE014F07013C24DB2D5
:10374B002D902041E030E50890201AE0A3F0D24DF7
:10375B00304E1B90201DE014F07013C24EB22E9011
:10376B002041E030E60890201CE0A3F0D24E304F11
:10377B001B90201FE014F07013C24FB22F9020410A
:10378B00E030E70890201EE0A3F0D24FE52A70034B
:10379B0002388E30501B902021E014F07013C25071
:1037AB00B230902042E030E008902020E0A3F0D22D
:1037BB005030511B902023E014F07013C251B231E2
:1037CB00902042E030E108902022E0A3F0D251306B
:1037DB00521B902025E014F07013C252B23290208D
:1037EB0042E030E208902024E0A3F0D25230531B89
:1037FB00902027E014F07013C253B233902042E0B4
:10380B0030E308902026E0A3F0D25330541B9020D5
:10381B0029E014F07013C254B234902042E030E42B
:10382B0008902028E0A3F0D25430551B90202BE0B9
:10383B0014F07013C255B235902042E030E5089079
:10384B00202AE0A3F0D25530561B90202DE014F027
:10385B007013C256B236902042E030E60890202C0E
:10386B00E0A3F0D25630571B90202FE014F0701AC3
:10387B00C257B237902042E030E70890202EE0A3E9
:10388B00F0D257E52B700302398530581B9020314D
:10389B00E014F07013C258B238902043E030E008C7
:1038AB00902030E0A3F0D25830591B902033E01415
:1038BB00F07013C259B239902043E030E1089020E8
:1038CB0032E0A3F0D259305A1B902035E014F0703F
:1038DB0013C25AB23A902043E030E208902034E011
:1038EB00A3F0D25A305B1B902037E014F07013C258
:1038FB005BB23B902043E030E308902036E0A3F02E
:10390B00D25B305C1B902039E014F07013C25CB2B8
:10391B003C902043E030E408902038E0A3F0D25CE8
:10392B00305D1B90203BE014F07013C25DB23D90F4
:10393B002043E030E50890203AE0A3F0D25D305E02
:10394B001B90203DE014F07013C25EB23E902043FA
:10395B00E030E60890203CE0A3F0D25E305F1B9095
:10396B00203FE014F07013C25FB23F902043E03071
:10397B00E70890203EE0A3F0D25F30020FD2018522
:10398B003E83853F82A385833E85823F200710C2FD
:10399B008CE58A2535F58AE58C3536F58CD28CD0BD
:1039AB0082D083D0E0D0D032C0D0C0E0C083C08200
:1039BB00C01F75D018209811309903023A87D01F79
:1039CB00D082D083D0E0D0D032C298E5874440F586
:1039DB0087309F2AC29F902100E0547FB40011745E
:1039EB0001F0E58754BFF587759840D29C023A09E0
:1039FB007400F0E58754BFF5877598C0D29CE587B6
:103A0B0054BFF587902100E0547FB40003023A3095
:103A1B00A3E0F58275835CE599F00582E582902140
:103A2B0001F0023A84902101E0F8A3E0F9A3E0FA57
:103A3B00A3E0FBE599FF309A1030E70DC29A7B01AA
:103A4B00E8FA0AEA6970027B00EB602175835C8AF5
:103A5B0082EFF00582E5826970047B00800FAA82F9
:103A6B000B309A098882EB14F0EAF87B0090210165
:103A7B00E8F0A3A3EAF0A3EBF00239C0C29910144B
:103A8B0003023A9121C0902200E0F8A3E0B5180C94
:103A9B00E4902203F0A3F0C2080239C0F890210091
:103AAB00E0547FB40031E8F8902204E07012758383
:103ABB005E8882E0902203F0902201E004F08011F6
:103ACB00F8902203E014B5180CE4902203F0A31431
:103ADB00F0D29B8002C29B902201E075835EF5823F
:103AEB00E0F5990582E582902201F0A3A3A3E004FF
:103AFB00F00239C0C0D0C0E0C0F0C083C08275D026
:103B0B0018753C01753D00753B00E53B9090052514
:103B1B0082F582E020E203023BE9C0E0902108E558
:103B2B003B2582F582E0FCA385823A858339547F5D
:103B3B00B4000E909001E53B2582F582E0A2E59260
:103B4B000C909003E53B2582F582E0F5F0EC20E745
:103B5B0003023BE7547FB40003023B87853A82851F
:103B6B003983E0F582E53D245DF583E5F0F00582D0
:103B7B00E582853A82853983F0023BE7853A828577
:103B8B003983E0FCA3E0FDA3E0FEA3E0FFE5F0300A
:103B9B000C1030E70DC20C7F01ECFE0EEE6D7002C7
:103BAB007F00EF60258E82E53D245DF583E5F0F027
:103BBB000582E5826D70047F00800FAE820F300CA2
:103BCB00098C82EF14F0EEFC7F00902109E53B2578
:103BDB0082F582ECF0A3A3EEF0A3EFF0D0E020E0AF
:103BEB0003023D26902208E53D2323232582F582FF
:103BFB00E0FFA3E0B51F22A3A37400F0A3F0909005
:103C0B0002E53B2582F58274B8F0909005E53B25E3
:103C1B0082F5827404F0023D26F5F085823A8583A5
:103C2B0039A3E0547FB400028008B407028003027A
:103C3B003D02C0E0A3E0FC600114FEA3E0FDD0E078
:103C4B00B40705BC00538003BC001FE5F0F582E50B
:103C5B003D245FF583E0FC0582E582853A82853958
:103C6B0083F0F5F0B51F07023C02EDB51E2B9090CB
:103C7B0002E53B2582F5827415F0909000E53B251B
:103C8B0082F582E0FEA3A37415F0909000E53B252E
:103C9B0082F582EE4404F08029909002E53B258268
:103CAB00F5827415F0909000E53B2582F582E0FEDD
:103CBB00A3A37415F0909000E53B2582F582EE549A
:103CCB00FBF0E5F0F582E53D245FF583E0FE058230
:103CDB00E582853A82853983F00DECB51D047C00B5
:103CEB007D00A3A3ECF0A3EDF0909003E53B2582C0
:103CFB00F582EEF0023D26E5F0F582E53D245FF519
:103D0B0083E0F5F00582E582853A82853983F09070
:103D1B009003E53B2582F582E5F0F0053DE53B247C
:103D2B0008F53BD53C028003023B15D082D083D0F3
:103D3B00F0D0E0D0D03216EA16EA15431549154FEC
:103D4B001555155B15F115F115F115F415FA1561EE
:103D5B00156D15A315A915AF15C115971579157FF8
:103D6B0015851591158B15C715CD15D315D915EBD4
:103D7B0015F115F115F116C016C61600160616D25A
:103D8B0016D8159D1573160C16121618161E16241A
:103D9B00162A1630165A16601666166C1672167898
:103DAB00167E1684168A16B416BA16CC15E516DED0
:103DBB0020CB21B7223A15DF16EA156715B515BBCF
:103DCB001636163C16421648164E16541690169674
:103DDB00169C16A216A816AE15F115F115F115F1D4
:103DEB0015F115F115F115F115F115F115F115F198
:103DFB0015F115F115F116E415F116EA16EA16EAA6
:103E0B0016EA16EA16EA0B494F36342056362E358B
:103E1B00330D0020494F36342076362E3533202093
:103E2B002020200020416C636F726E204D63427224
:103E3B0069646520002053686F7720646174613A70
:103E4B002062616420002053686F77206461746185
:103E5B003A20206F6B200020466C61672042616E18
:103E6B006B20232031202020466C61672042616E3D
:103E7B006B20232032202020466C61672042616E2C
:103E8B006B20232033202020466C61672042616E1B
:103E9B006B2023203420205374617465205661728B
:103EAB006961626C65202357616974696E6720666E
:103EBB006F72202020202020202020202020202056
:103ECB002020202020202020202020202020200007
:103EDB0065787465726E616C2073796E632E2E2E0D
:103EEB0020202020202020202020202020202020C7
:103EFB0020202020202020200045787465726E61E0
:103F0B006C2073796E63202020202020202020201D
:103F1B002020202020202020202020202020202096
:103F2B0020007265636F76657265642E20202020F9
:103F3B002020202020202020202020202020202076
:0B3F4B0020202020202020202020002B
:00000001FF
